:020000040000FA
:040000008A01152834
:06002A0083160313FF30F2
:100030008500860108309B009F019F1783120313E0
:100040009F151F169F121F139F131F143D2083120D
:1000500003131F151F192A28831603131E08831262
:10006000031386006C201E0886006C2027280000E1
:100070000000000000000000000008000000A430A4
:100080004A28000040304A281F304A2800000E301D
:100090004A280530A000A00B4B280800C8305D2876
:1000A00064305D2832305D2814305D280A305D28C8
:1000B00005305D2802305D280130A100F930A00034
:1000C0000000A00B6028A10B5E280800C830712832
:1000D0006430712832307128143071280A30712848
:1000E0000530A2006430A100F930A0000000A00B90
:0C00F0007628A10B7428A20B72280800CF
:00000001FF
